:100000000C949E010C94BB010C94D6010C94BB0182
:100010000C94BB010C94BB010C94AB160C94BB016B
:100020000C94BB010C94BB010C94BB010C94BB0160
:100030000C94BB010C94BB010C9487160C94BB016F
:100040000C94BB010C94BB010C94BB010C94BB0140
:100050000C94BB010C94BB010C94BB010C94BB0130
:100060000C94BB010C94BB010000000000000000D8
:100070000000000000000000000000000000000080
:100080000000000000000000000000007E0F00D40F
:10009000FFFFFFC700000078000000000000000024
:1000A0002A2B2800000000000000000000000000D3
:1000B00000000029000000002C1E342021222434DE
:1000C0002627252E362D3738271E1F2021222324B0
:1000D00025263333362E37381F0405060708090A4C
:1000E0000B0C0D0E0F101112131415161718191AE8
:1000F0001B1C1D2F3130232D350405060708090A66
:100100000B0C0D0E0F101112131415161718191AC7
:100110001B1C1D2F3130354C530054005500560028
:100120005F006000610000005C005D005E00570041
:1001300059005A005B000000620000006300580094
:1001400001000100010001000100010001000000A8
:100150000100010001000100010001000100000098
:100160000100000001000100010001000100010088
:100170000100010001000000010001000100010078
:100180000100010001000000010000000100010069
:100190000100010001000100010001000100000058
:1001A0000100010001000100010001000100000048
:1001B000010000000100010005010902A101850202
:1001C0000901A10005091901290815002501950853
:1001D000750181020501093009311581257F9502DC
:1001E0007508810609381581257F950175088106F6
:1001F000050C0A38021581257F950175088106C016
:10020000C005010980A101850319012AB700150164
:1002100026B700950175108100C0050C0901A101E8
:10022000850419012AA002150126A0029501751066
:100230008100C00660FF0961A1010962150026FF67
:10024000009520750881020963150026FF0095209E
:1002500075089102C005010906A101050719E029E9
:10026000E715002501950875018102950175088142
:10027000030507190029FF150026FF0095067508DC
:10028000810005081901290595057501910295015F
:1002900075039103C0120344004900530043004911
:1002A000005000410044000000200363006F007311
:1002B0000065007900660061006E006E00690074E0
:1002C000007500740074006900000004030904094B
:1002D000025B00030100A0320904000001030101D8
:1002E00000092101010001224000070581030800E7
:1002F00001090401000203000000092101010001BD
:1003000022220007058403080001070504030800F2
:10031000010904020001030000000921010100019C
:10032000227B000705830308000112011001000071
:100330000008626B691701000102000111241FBE51
:10034000CFEFD8E0DEBFCDBF22E0A8E4B1E001C02E
:100350001D92A43DB207E1F711E0A0E0B1E0ECE1AD
:10036000F7E302C005900D92A834B107D9F70E94B7
:10037000D2160C946D1B0C940000A82FB92F80E0AE
:1003800090E041E050EA609530E009C02D9182276D
:100390009795879510F084279527305EC8F36F5F97
:1003A000A8F30895EADF8D939D930895CF93CFB777
:1003B000CF93DF93C3954B9BE9F74B9B10C04B9BAF
:1003C0000EC04B9B0CC04B9B0AC04B9B08C04B9B69
:1003D00006C0C091AE02C395C093AE028EC06F93AB
:1003E000C091AD02DD27CE54DD4F2F9365E54B9BC9
:1003F00003C02F916F91E1CF0F931F934F9320E094
:1004000040E15F9309B10C7003FB27F93F9350E083
:100410003BE039C01C7040642F77012F5F5F1EC026
:10042000406819B11C702F7752501FC0406409B149
:100430002F770C70D1F15F5F00C023C0406219B10B
:100440002F771C7091F15F5F00C025C00C701027E2
:10045000515012F45D5F0000115027952C3F19B1E7
:10046000C8F61C700127015027952C3FC8F642277B
:10047000499309B10C7010274F73115027952C3FE9
:10048000A8F64695469519B11C7079F001270150E0
:1004900027952C3F98F66B5A60F3315009B1B0F6AE
:1004A00000C012E01CBB00271CC03B503195C31B91
:1004B000D04012E01CBB0881033C21F10B3411F148
:1004C0002091AB021981110F1213EDCF4A81441F05
:1004D000093679F10D3211F0013E29F74F7009F01C
:1004E000042F0093B1023F915F914F911F910F91A3
:1004F0002F916F91CCB3C1FD5DCFDF91CF91CFBF75
:10050000CF9118952091B102222369F31091AF0287
:10051000112309F049C034300AF448C03093AF02C7
:100520002093AC021091AD023BE0311B3093AD0241
:100530003DC00091AF020130BCF50AE54F7049F4AF
:1005400030910D0134FD33C000930D01C8E8D2E0B5
:1005500032C0433059F0443091F03091930234FD71
:1005600026C000939302C4E9D2E025C03091C802AE
:1005700034FD1DC00093C802C9ECD2E01CC030910C
:100580009F0234FD14C000939F02C0EAD2E013C062
:10059000052710E000C000000BB91AC0052710E0C5
:1005A000221F1DC010E021C04AE502C032ED432FDA
:1005B000C4E1D0E032E01AB11C605B9A0BB11AB909
:1005C0005CE020E865E320FF05270BB92795179528
:1005D0001C3FF0F66695B8F7B1F720FF05270BB979
:1005E000279517951C3FD0F62795179517FF0527D8
:1005F00000001C3F0BB9B0F629913A9519F7037F1B
:100600001091B002110FC651D0400BB911F01093E8
:10061000AB0212E01CBB08601AB1137F402F437F6E
:1006200054E05A95F1F70BB91AB94BB95CCFFC01FC
:100630008381833089F130F48130F1F0823021F10F
:1006400080E00895813209F441C08232C9F72481E3
:1006500035812130310509F457C02115310509F4E0
:100660004BC02230310561F788EB91E09093830213
:10067000809382028BE708958AE293E0909383024D
:100680008093820282E108958FEC92E0909383023E
:10069000809382028BE508958281813079F08823EE
:1006A00029F0823069F685E992E0E8CF8BEC92E0A0
:1006B000909383028093820284E0089589EA92E015
:1006C000909383028093820280E208958281813038
:1006D00081F0882331F0823009F0B2CF8AE193E0D3
:1006E00002C081EE92E0909383028093820289E0BF
:1006F00008958AEF92E0F7CF85E592E09093830228
:100700008093820280E4089523E332E030938302F1
:10071000209382020895089580917D02089588E1D2
:1007200098E00FB6F894A895809360000FBE909360
:100730006000A895F894D8E0CEEF28E3299320E054
:10074000299314BEFFCF08959C014FB7F894809170
:10075000C6019091C701A091C801B091C9014FBFD6
:10076000821B930B08952FB7F8948091C601909146
:10077000C701A091C801B091C9012FBF0895209170
:10078000C2013091C3012817390771F09093C3015A
:100790008093C201E091C001F091C101309721F036
:1007A0000084F185E02D099508952091BE013091D6
:1007B000BF012817390771F09093BF018093BE01E4
:1007C000E091C001F091C101309721F00680F781DE
:1007D000E02D09950895E091C001F091C101309795
:1007E00029F00190F081E02D0995089580E00895A9
:1007F0000E94B3039C019091BA018091BB01982B98
:1008000021F03093B7012093B6019091BC01809103
:10081000BD01982B21F03093B5012093B401E091F4
:10082000C001F091C101309749F082E08093B80196
:100830000480F581E02D88EB91E0099508954091C1
:10084000BA01803F59F48091BB0187FF0DC010921F
:10085000BB0141110BC01092B20108C0813F81F46D
:100860008091BB0118169CF3442381F08091BC0158
:100870009091BD01892B09F05AC01092B1010895E1
:10088000823F49F447FFF0CF1092BA018091BB013B
:100890008111ECCFE0CF833F19F41416ACF3E4CF11
:1008A0009091BC01893F29F41916F4F61092BC010D
:1008B000DBCF8A3F19F497FFD7CFF8CF9091BD01D6
:1008C0008B3F29F497FFD0CF1092BD01CDCF8C3F45
:1008D00019F41916CCF3C8CF9CE0980F953090F41A
:1008E000845F990B21E030E0B90102C0660F771FE9
:1008F0008A95E2F7CB0180959091B9018923809385
:10090000B901B2CF8D3F31F48091B3018E7F8093D6
:10091000B301AACF8E3F21F48091B3018D7FF7CF31
:100920008F3F09F0A1CF8091B3018B7FF0CF089565
:100930008091B30180FD16C081FD16C082FD16C0F6
:100940008091B1018823A1F0883280F428E0829F51
:10095000C001112468E270E00E94B21A862F672B52
:1009600039F0089582E0089584E0089588E00895BC
:1009700081E008958091B30180FD14C081FD14C011
:1009800082FD16C08091B201882381F08E3180F4FF
:1009900020E5829FC00111246EE170E00E94B21A2E
:1009A000862F089584E1089588E2089588E00895E7
:1009B00080E50895803F31F40E94BA0481958093C8
:1009C000BB010895813F19F40E94BA04F8CF823F19
:1009D00031F40E94BA0481958093BA010895833F4F
:1009E00019F40E94BA04F8CF893F29F40E949804B0
:1009F0008093BC0108958A3F21F40E949804819558
:100A0000F7CF8B3F31F40E94980481958093BD010C
:100A100008958C3F19F40E949804F8CF9CE0980F39
:100A2000953070F4845F990B21E030E001C0220F13
:100A30008A95EAF78091B901822B8093B9010895D4
:100A40008D3F31F48091B30181608093B3010895AB
:100A50008E3F21F48091B3018260F7CF8F3FB9F7C9
:100A60008091B3018460F1CF80E00895F894E82F7D
:100A7000E295EF70F0E031A1282F2F7081E090E037
:100A800001C0880F2A95EAF7982F9095932391A398
:100A900092A1892B82A3789408959091A10192FF4D
:100AA00006C0282F28712830F9F4877F846093FFCF
:100AB00006C0282F28712831F1F4877E84612091A7
:100AC000A20120FF06C0382F38713830D9F4877F53
:100AD000816021FF06C0282F28712831D1F4877E3C
:100AE000816194FD877E0895282F24712430F9F6C2
:100AF0008B7F8860DCCF282F2471243101F78B7E17
:100B00008861DDCF382F3171313019F78E7F8860E1
:100B1000E0CF282F2171213121F78E7E8861E1CF2E
:100B2000CF93DF93EC0182389105A9F1D8F5813399
:100B3000910509F496C048F58932910509F48AC0F7
:100B40008A9709F495C0C11521E5D20708F0BCC009
:100B5000C11530E5D30708F014C1C83ED10508F02F
:100B60009CC0C03ED10560F5C83AD10508F087C0E9
:100B7000C53AD10508F0FDC0C130D10509F1209773
:100B8000F9F0C430D105E0F440C08533910509F493
:100B90005AC0C997C1F68091A101837089F0C0EE57
:100BA000D0E00EC0833E910599F170F4803E91052E
:100BB00001F1823E910539F68091A10182FD21C0AB
:100BC000CE01DF91CF910895863E910561F1873E78
:100BD000910571F1843E910509F0B5CF8091A20194
:100BE00081FFEECF8091A101C7EED0E084FD0DC062
:100BF000E7CF8091A10180FD12C19091A20190FFE9
:100C0000DFCFC3EED0E084FFDBCFD0E0C0E0D8CFB1
:100C10008091A10182FD06C19091A20190FDBFCFFC
:100C200084FFCECFF2CF8091A10183FDDDCFC8CF6D
:100C30008091A10183FDF9C09091A20191FFF0CFB5
:100C4000C4EED0E0BDCF8091A10185FFB9CFC9E24C
:100C5000D0E0B6CF8091A10185FFB2CFC5E3D0E04F
:100C6000AFCF8091A10186FFABCFCAE2D0E0A8CF81
:100C70008091A10186FFA4CFC1E3D0E0A1CFCF3BFB
:100C8000D10518F6C85AD0E0CC0FDD1FCF5EDE4F7D
:100C90000990D881C02DD46493CFC11540E2D40708
:100CA00058F4C11581E0D80708F08ACFC03FD105BC
:100CB00008F4ABCFD06584CFC11590E4D90708F410
:100CC000A4CFDF70D06A7CCFC11525E5D20700F52F
:100CD000C11534E5D30708F08AC0C11543E5D40730
:100CE00008F071C0C11582E5D80708F467C0CE01CD
:100CF0008370992721E030E002C0220F331F8A95CC
:100D0000E2F7C695C69580E2C89FE001112452C063
:100D1000C11599E5D907A8F4C11528E5D20708F04F
:100D20006BC0C11536E5D30708F06FCF8C2F0E943A
:100D30004D05C82FD0E0DC2FCC27CC27DF71D06247
:100D40003FCFC1154AE5D40708F45BC0CE019056E9
:100D50008115904208F059CF8D2F8F710E944D055B
:100D600090E0982F882788279F719C012C2BE90100
:100D7000E6CFC55AD0E0C25FDE4FC881D0E0D06474
:100D80001FCFCE01E4E096958795EA95E1F7837051
:100D90002C2F26952695237040E2249F9001112444
:100DA000382B8C2F8370C1E0D0E002C0CC0FDD1F48
:100DB0008A95E2F7C22BD32BDC6802CFDC2FCC273D
:100DC000C16FD06AFDCECE018370992721E030E05B
:100DD00002C0220F331F8A95E2F7C695C69590E2AE
:100DE000C99FE0011124C22BD32BDA68E9CEDC2F96
:100DF000CC27C46FD06AE4CEDC2FCC27C06FD06A7A
:100E0000DFCE8C2F8F700E944D0534E0D695C795AC
:100E10003A95E1F7CF709C2FEC01D069D1CEC9E3B0
:100E2000D0E0CECEC2EED0E0CBCEC6EED0E0C8CE83
:100E3000809197018111109297010895809590916A
:100E40009601982390939601089580919601909130
:100E50009501892B80934A0190919701992391F0F4
:100E6000892B80934A0120E08CE491E0FC013191D0
:100E7000CF0131112F5FF1E082359F07B9F72111C2
:100E80000E941807E091C001F091C101309731F044
:100E90000280F381E02D8AE491E009950895ECE465
:100EA000F1E09191891303C0DF0111971C9291E049
:100EB000E235F907B1F70895ACE4B1E0EFEF90E067
:100EC0002D91821751F0EF3F19F4211101C0E92F44
:100ED0009F5F9630A9F7EF3F09F408950E2E000C9E
:100EE000FF0BE65BFE4F8283089580919301909102
:100EF0006201981301C008958F5F8770FACF953013
:100F000080F5843070F544E0949F90011124820FA5
:100F1000932F911D682F677023E0969587952A95EA
:100F2000E1F7FC01EE0FFF1FE80FF91FED5AFE4F2E
:100F300050E040E080E0219130E0062E02C036957E
:100F400027950A94E2F721703327042E01C0220F5F
:100F50000A94EAF7822B4F5F5F4F4330510559F7F0
:100F6000089580E00895953098F5843088F544E040
:100F7000949F90011124820F932F911D282F277089
:100F800041E001C0440F2A95EAF723E09695879542
:100F90002A95E1F7FC01EE0FFF1FE80FF91FED5A4C
:100FA000FE4F90E080E070E05191DF0111979B01CE
:100FB000082E02C0369527950A94E2F721702195F4
:100FC0002527242325272C9301968330910561F74B
:100FD000089590E080E00E94D50390E080E00E94B8
:100FE000BF03109295010E94250786E0E8EBF1E02F
:100FF000DF011D928A95E9F71092B2011092B101BA
:101000001092B3010E94F8030895809387020E9412
:10101000E907089580918702982F9670963021F401
:1010200088600E9405080895877FFBCF21E030E0AB
:1010300001C0220F8A95EAF72095809187028223CA
:101040000E940508089590919401809589238093CA
:101050009401282F277091F4282F082E000C330BB1
:101060009217130659F09091A20192FF07C085953F
:10107000859585950E94160810929401089521E0A7
:1010800030E001C0220F8A95EAF780918702822B17
:101090000E9405080895809398010E94E907089529
:1010A000882321F00E941E070E94250708958823A7
:1010B00039F090919601982B909396010E94250704
:1010C0000895882309F455C0823879F40E94EB030F
:1010D00081FF4FC089E30E945C070E94250789E3D6
:1010E0000E944F070E9425070895833859F40E94F3
:1010F000EB0380FF3EC083E50E945C070E9425074A
:1011000083E5EECF843859F40E94EB0382FF31C0AF
:1011100087E40E945C070E94250787E4E1CF9CEFEB
:10112000980F913AE8F290E2980F983050F4877057
:1011300091E001C0990F8A95EAF7892F0E941E0756
:10114000D1CF9BE5980F933028F490E080E00E9487
:10115000D503089598E5980F973128F490E080E042
:101160000E94BF030895803F20F00E941F040E9448
:10117000F80308958091C501882321F11092C401DC
:1011800088E190E020E40FB6F894A8958093600081
:101190000FBE2093600083B7817F846083BF83B7D5
:1011A000816083BF7894889583B78E7F83BF0FB6A5
:1011B000F894A895809160008861809360001092F7
:1011C00060000FBE0895CF93DF938091AF028350EC
:1011D00087FD14C09091AD02CCE0D0E0C91BD109CD
:1011E000CE54DD4F9091AC02903108F06BC0883046
:1011F00009F453C0109272021092AF0280910D0157
:1012000084FF3EC080910C018F3FD1F1C82F8930FF
:1012100008F0C8E0982F9C1B90930C0190918802D5
:1012200028E89227909388028823E9F0809182022F
:10123000909183022091810226FF06C1FC012C2F90
:10124000A9E8B2E034913D9331962150D9F79C0141
:101250002F5F3F4F8FEF8C0F820F932F911D909335
:101260008302809382026C2F89E892E00E94D2016F
:10127000CC5FCC3019F08FEF80930C01C0930D013F
:1012800084E199B19C7031F48150D9F71092B00289
:101290001092AB02DF91CF91089580917202893153
:1012A00008F0A8CFE82FF0E0EE5AFD4F9E01285F2E
:1012B0003F4F99919193C217D307D9F7885F8093D5
:1012C00072029ACF9D3209F0A3C0883009F094CF02
:1012D00083EC809388028AE580930D01109281024D
:1012E0008881807609F447C0803229F58981813070
:1012F00099F48C819D81892BF1F484E792E090939D
:1013000083028093820288E09F81911131C09E8187
:10131000981770F5892F2CC0823041F483E792E052
:10132000909383028093820281E0EECF8A3029F489
:101330008B818093730280E0E7CF8930E1F78A8167
:101340009B818115924069F48C819D81892B49F4A0
:1013500081E0809380028E819F8190937F028093B1
:101360007E02888187FF52C08E8190E8909381022F
:1013700080930C0141CF2A811092910299819111A1
:101380000AC01092920221E932E082E03093830297
:1013900020938202B9CF953029F42093B00221E93D
:1013A00032E0F4CF9630C1F49B81913049F4CE0104
:1013B0000E94170390E4909381028F3F91F2A4CF93
:1013C0009230A9F3933099F3913289F3923279F301
:1013D00090E49093810298CF983089F0993019F475
:1013E00020937C02DCCF9A3071F09B30C1F69BE4F5
:1013F000909394029093C9029093A002D0CF2CE7CF
:1014000032E081E0C3CF21E932E0FBCF8FEFADCFF7
:101410008091810287FFF0CE80917E0290917F02C1
:10142000892B71F080918002813051F48881809302
:101430007D0210927F0210927E0210920C01DCCE8F
:101440008EE180930D01D8CEDC012C2FE9E8F2E08B
:101450003D9131932150E1F7FACE1F93CF93DF9363
:10146000E82F792F162FEA01888184FF1CC029817B
:1014700088E828272983CE010296DC012E2F372FFA
:10148000512F5E0FF90121912D939F01452F4E1B86
:101490001416C4F3612F0E94D2011C5F1883DF91E0
:1014A000CF911F9108958AE58883E5CF2091C802E6
:1014B00024FF05C048EC52E066E00E942D0A089522
:1014C00090915102981307C020914F023091500221
:1014D00026173707B9F0809351027093500260933A
:1014E0004F0280934C0270934E0260934D028091A4
:1014F000C80284FF07C048EC52E063E08CE492E04D
:101500000E942D0A0895BC0184E00E94600A08959B
:10151000BC0183E00E94600A0895CF93DF93CAE084
:10152000D0E08091930284FF1CC080914A02909188
:101530004B02981799F028E0829FC001112443E9DB
:1015400052E068E086539E4F0E942D0A80914A0225
:1015500090E001968F70992780934A02DF91CF9196
:1015600008950E94E3088FE99FE00197F1F700C01A
:1015700000002197B1F6F2CFCF93DF93EC01A09159
:101580004B02B0E0CD0101968F70992720914A025D
:10159000281779F093E0AA0FBB1F9A95E1F7A6539D
:1015A000BE4F98E0FE0101900D929A95E1F780936D
:1015B0004B020E94E3080E948D0A88E0FE01A4E726
:1015C000B2E001900D928A95E1F7DF91CF910895F5
:1015D000CF93C82F8823C9F08238C9F40E94EB0347
:1015E00081FD13C089E30E945C070E9425072FEF4D
:1015F00081EE94E0215080409040E1F700C000006F
:1016000089E30E944F070E942507CF9108958338F0
:10161000A1F40E94EB0380FDF8CF83E50E945C07F4
:101620000E9425072FEF81EE94E0215080409040EA
:10163000E1F700C0000083E5E4CF8438A1F40E9404
:10164000EB0382FDE2CF87E40E945C070E9425073E
:101650002FEF81EE94E0215080409040E1F700C0F0
:10166000000087E4CECF8CEF8C0F813A68F4ECE475
:10167000F1E08191C817E1F121E0E235F207C9F705
:101680008C2F0E945C07BFCF80E28C0F883068F4FB
:10169000C77021E030E001C0220FCA95EAF78091BF
:1016A0009601822B80939601AECFEBE5EC0FE330F1
:1016B00040F4F0E0E25FFE4F808190E00E94D503AD
:1016C000A4CFE8E5EC0FE73150F4F0E0EE0FFF1F98
:1016D000EF5EFE4F808191810E94BF0396CFC03F95
:1016E00008F493CF8C2F0E94DA040E94F8038DCF68
:1016F0008C2F0E944F070E942507C2CF1F93CF93C4
:10170000DF93182FD0E0C0E0893311F4C0E5D0E0BA
:10171000812F0E94E80A209739F4812F0E946108E6
:10172000DF91CF911F9108958FE99FE00197F1F725
:1017300000C000002197EFCF0F931F93CF93DF934B
:10174000C62FD42F022FFC0182818823A9F0609339
:1017500086020E94B3039093850280938402C7702F
:1017600081E001C0880FCA95EAF70E945708DF910F
:10177000CF911F910F91089580918602681332C016
:1017800080918402909185020E94A403883C910577
:1017900048F510E21D0FCD17B9F080E28C0F8830AC
:1017A00040F4C77081E001C0880FCA95EAF70E9433
:1017B0005008183048F481E09D2F977001C0880FC1
:1017C0009A95EAF70E945708802F0E947E0B1830E6
:1017D00070F6D77081E001C0880FDA95EAF70E94B1
:1017E0005008C5CFC77081E001C0880FCA95EAF7DD
:1017F000F6CFCF93DF93C7ECD0E060E0CE010E943C
:10180000391B2196C11584E0D807B9F7DF91CF9134
:1018100008951F93CF93DF93122F8430E0F4653047
:10182000D0F44430C0F498E0699FE001112450E006
:10183000440F551FC40FD51F98E2899FC00DD11DBD
:101840001124632FCE0187960E94391B612FCE0190
:1018500088960E94391BDF91CF911F910895AF9216
:10186000BF92CF92DF92EF92FF921F93CF93DF93BD
:1018700088E1C82E81E0D82ED0E07601C0E014C007
:10188000F50125913491412F6C2F8D2F0E94090C69
:1018900082E0A80EB11C1F5F143091F788E0E80EBB
:1018A000F11CCF5FC53019F0570110E0E9CFDF5FC1
:1018B00088E2C80ED11CD43001F7DF91CF911F917F
:1018C000FF90EF90DF90CF90BF90AF900895CF93AF
:1018D000C82F6FEF811162E283E290E00E94391B12
:1018E0006FEFC11164E084E290E00E94391B6FEF5A
:1018F000C11163E185E290E00E94391BCF91089508
:1019000080E00E94670C60E086E290E00E94391B54
:101910000E942F0C0E94F90B81E00E94670C089531
:10192000CF93C091A201C2FB992790F9981791F02B
:1019300080FBC2F9C093A2016091A10184E090E014
:101940000E94391B6C2F82E290E00E94391B82E0DA
:101950000E942308CF9108950F931F93CF93DF9395
:10196000843030F5653020F5443010F528E0629F72
:101970008001112450E0440F551F040F151F38E259
:10198000839F000D111D1124C80187960E942B1BF7
:10199000C82FD0E0DC2FCC27C80188960E942B1BD3
:1019A0009E01282BC901DF91CF911F910F910895BE
:1019B00090E080E0F8CF462F843040F4753030F46A
:1019C000643020F4672F0E94AC0C089590E080E012
:1019D0000895CF92DF92FF920F931F93CF93DF93DF
:1019E0006C010091870280919801082BC7E0D0E03C
:1019F00010E0FC2EC8010C2E02C0959587950A9424
:101A0000E2F780FD0CC02197A0F7F12C8F2DDF911C
:101A1000CF911F910F91FF90DF90CF900895B60165
:101A20008C2F0E94DB0C0E949005019761F3EECF92
:101A3000CF93DF93EC010E94E90CBE010E94DB0C06
:101A40000E949005DF91CF910895FC0180819181E2
:101A50000E94180D92959F70963091F058F4925F05
:101A60009F70923058F4803F19F030F4883E30F483
:101A700081E008959A5FF4CF843FD1F380E0089528
:101A8000883EB0F3813FD1F7F3CF83E290E00E942C
:101A90002B1B823289F484E290E00E942B1B84305D
:101AA00059F485E290E00E942B1B91E0833109F00C
:101AB00090E0892F8170089580E0FCCFCF9384E07F
:101AC00090E00E942B1BC82F82E290E00E942B1B0B
:101AD000982F8C2FCF910895A5E0B0E0E2E7FDE0CC
:101AE0000C94DA1A8E010F5F1F4F85E0F8011192F6
:101AF0008A95E9F78FE3C82E81E0D82EF12CE12CEE
:101B0000AA24A394B12CF60181916F018F3F09F4AF
:101B100043C0F894E82FE295EF70F0E021A18F70B8
:101B2000A50102C0440F551F8A95E2F7CA01922F02
:101B3000982B91A392A18095892382A3789400C0C9
:101B4000E4E4F1E0912C31E021912F3F09F46AC0E7
:101B5000A22FA295AF70B0E090968C9190E02F707C
:101B600002C0959587952A95E2F780FD5BC0832F8B
:101B7000982A330F51E0E834F50731F7F601319731
:101B800080818F3F11F00E94360580EA8A95F1F737
:101B9000F801EE0DFF1D9082EFEFEE1AFE0AF5E060
:101BA000EF16F10409F0AFCF45E050E0B8018CE941
:101BB00091E00E941E1BFF24F394009709F4F12C7E
:101BC000892B91F185E0F801ACE9B1E001900D922B
:101BD0008A95E1F781E080939B010E94B303909383
:101BE0009A01809399018091990190919A010E94A4
:101BF000A4030597E8F080919C018093AA0180914D
:101C00009D018093AB0180919E018093AC018091F6
:101C10009F018093AD018091A0018093AE0110924D
:101C20009B0106C080E0A4CF80919B018111DBCF96
:101C30008F2D2596EBE00C94F61A10929601ECE4A9
:101C4000F1E086E0DF011D928A95E9F70E94E9073D
:101C500008950E941D0E2FEF84E39CE021508040E8
:101C60009040E1F700C0000088E198E00FB6F894DA
:101C7000A895809360000FBE90936000FFCF68EE40
:101C80007EEF90E080E00E94571B60E082E090E0F1
:101C90000E94391B60E083E090E00E94391B1092A3
:101CA000980160E084E090E00E94391B64E082E2E9
:101CB00090E00E94391B60E085E090E00E94391BB3
:101CC00060E086E090E00E94391B6FEF87E090E0D3
:101CD0000E94391B40E050E0BA0188E090E00E9489
:101CE0004B1B60E08DE090E00E94391B40E050E02B
:101CF000BA0188E190E00E944B1B60E087E190E030
:101D00000E94391B40E050E0BA018CE190E00E9453
:101D10004B1B70E060E080E290E00E94571B40E0C7
:101D200050E0BA0188E190E00E944B1B80E00E94E5
:101D3000670C0E94800C40E050E0BA018FE090E018
:101D40000E944B1B40E050E0BA0183E190E00E940A
:101D50004B1B0895A5E0B0E0E0EBFEE00C94D41A34
:101D60008C01FC0183819481892B31F080819181E8
:101D700089238F3F09F04EC52596E1E10C94F01AB6
:101D80000E94E90CF82E682F89819A810E94B3077E
:101D900069817A818F2D0E94DB0C7C01F8018281A0
:101DA000882309F4FDC4970122513F4520313105B4
:101DB00008F023C58FEF93E00E942B1B811127C0F1
:101DC000FEEEEF0E57EC852E912CE11032C01C82F6
:101DD0001B82442443944AE0342E74018FEFE81AA6
:101DE000F80AC4010E942B1B89831A82882379F088
:101DF0009FEF980F933058F58A83498292E0890EBD
:101E0000911CC7010E942B1B8B83811121C08091E3
:101E10009401877009F4B0CFF8018281882309F416
:101E2000ABCF8091A20182FFA7CF82E00E9423085E
:101E3000A3CF811424E0920651F3C4010E942B1B0E
:101E4000811101C0EA943FEF831A930ABECF470184
:101E5000FE0131967F01F7012081222309F4BDCFD5
:101E6000213009F047C091818281913031F4F2E054
:101E7000EF0EF11C0E947E0B07C0923049F422E065
:101E8000E20EF11C0E94E80A3FEFE31AF30AE3CFE7
:101E9000933031F432E0E30EF11C0E946108F4CF7C
:101EA000943021F08FEFE81AF80AEECF92E0E90EB5
:101EB000F11C30E020E0B7016F5F7F4FF7014181F7
:101EC0008053990B8A30910550F021503109E0F28E
:101ED0008FE99FE00197F1F700C00000F6CF329E36
:101EE000F001339EF00D11249C012E0F3F1F842F13
:101EF0007B01E1CFE22FF0E0E856FF4F5490822FB4
:101F000086958695869590E0FC01E857FF4F649092
:101F10002770712C022E02C0759467940A94E2F720
:101F2000E1E06E227724FC01E858FF4FA490B12C29
:101F3000022E02C0B594A7940A94E2F7F1E0AF2212
:101F4000BB24FC01E859FF4FC490D12C02C0D594AA
:101F5000C7942A95E2F721E0C222DD2461147104BE
:101F600019F081EE0E94E80AA114B10419F086EE7E
:101F70000E94E80A852D0E947E0BA114B10419F07D
:101F800086EE0E9461086114710419F081EE0E94CE
:101F90006108C114D10409F477CF8CE26BCF81E0E2
:101FA0000E943F080E940A0832CF81E00E94160872
:101FB000F9CF82E0FBCF95EFE9169CE5F90609F42D
:101FC0006CC008F466C027E245EE66EEF6EFEF1649
:101FD000FCE5FF0609F40DC4882309F42CC4109213
:101FE000860223E0E2162DE5F20608F05DC03AEF26
:101FF000E3163CE5F30630F4C70182509C45449754
:1020000008F05EC00E945E0D9093A2018093A10132
:10201000E1E1EE16ECE5FE0609F436C108F0A4C0D5
:1020200029E0E2162CE5F20609F41CC108F06DC0A7
:1020300085E0E8168CE5F80609F408C108F056C0FA
:10204000E3E0EE16ECE5FE0609F4F6C008F0FAC08F
:102050008091A101816022E0E2162CE5F20609F4EC
:10206000EEC06091A101F090A20184E090E00E9496
:10207000391B6F2D82E290E00E94391B0E941D0ED9
:10208000C6CE27E245EE65EEB4C326E241EE60EE31
:10209000B0C327E245EE64EEACC326E241EE62EE49
:1020A000A8C328E241E0EFCF81E6E8168DE5F80607
:1020B00009F4A8CF95EAE9169DE5F90609F4A2CF3F
:1020C00036E1E3163CE5F30609F0C3C380919601BF
:1020D0008A7A91E009F490E090935201811102C153
:1020E00089E20E945C070E94250791CE8091A101A0
:1020F000806237E0E3163CE5F30609F4A0C008F47B
:10210000ADC08091A10180649AC08091A1018B7FB4
:102110009DE0E9169CE5F90609F491C0B0F48091C0
:10212000A1018E7FFBE0EF16FCE5FF0609F487C0F6
:102130008091A1018C602CE0E2162CE5F20608F4F7
:102140007EC08091A1018D7F7AC08091A1018F7E98
:102150003FE0E3163CE5F30609F471C008F488C0DB
:102160008091A1018F7D6BC09DEFE9169CE5F9067A
:1021700009F486C078F5F5E1EF16FCE5FF0609F4F1
:1021800091C0A0F48091A101837F33E1E3163CE587
:10219000F30609F454C008F47BC00E941D0E909110
:1021A000A101892F97FB87F9805849C09BEFE91659
:1021B0009CE5F90609F44EC008F05EC08091A201CA
:1021C0008160FAEFEF16FCE5FF0609F04ACF809335
:1021D000A20147CF21E0E2162DE5F20609F46EC018
:1021E000B8F48FEFE8168CE5F80609F457C0809133
:1021F000A2018360E1149DE5F90648F38091A201F4
:10220000982F909591708E7F892B90FB81F9DFCF6D
:10221000E1E6EE16EDE5FE0609F456C0F5EAEF1626
:10222000FDE5FF0609F457C022E0E2162DE5F206AF
:1022300009F017CF60E043C08091A10182608093D4
:10224000A1010FCF8091A1018460F9CF8091A101FC
:102250008860F5CF8091A2018260B9CF8091A10101
:102260008061EDCF0E941D0E8091A1018068E7CFB3
:102270008091A101877FE3CF8091A2018E7FA7CFBC
:102280008091A2018D7FA3CF8091A1018F7BD7CFB9
:102290000E941D0E8091A1018F77D1CF8091A20164
:1022A0008C7F95CF8091A10182FB992790F921E045
:1022B000922790FB82F990FB83F9C1CF61E08EE019
:1022C00090E00E94391BCDCE9091A101892F8F7E85
:1022D00094FF8061B4CF9091A101892F8E7F90FFF0
:1022E0008160ADCF85E3FDCE85E3B0C20E941D0EB7
:1022F0008FEF94E3ECE081509040E040E1F700C0C4
:1023000000000E948F0383CD8091A20182FB882769
:1023100080F991E089270E94900CF8018281E08089
:10232000F180882309F445C0C7010E94E90CD82E2A
:10233000682FC7010E94B307B7018D2D0E94DB0CE7
:102340000E9490057C01882EF801D280B580B2945D
:102350003FE0B322809194018770C1F0AD2CDD2065
:10236000B1F08F2D807F803421F080E28E0D883097
:1023700068F08091A20182FF09C082E00E942308D8
:10238000809194018770AA24A3948111A12C9F2C81
:1023900092942FE09222FBE0F91508F479C0E92D20
:1023A000F0E0E159F44E0C94C61A81E0B4CF80E01D
:1023B000B2CFC7010E947F07D82EBECF2F2D2F701E
:1023C000C22E8F2D807F19F0C29490EFC922DD209C
:1023D000B9F0CC2069F080E28E0D883010F08110C9
:1023E00009C080919601C82AC09296010E942507D3
:1023F0008E2D4CC080919501C82AC0929501F6CFD0
:102400008E2D0E946108CC2009F442C080E28E0D1E
:10241000883010F0811004C08C2D0E941E0706C069
:10242000C09480919501C822C09295010E94250711
:102430002FC03F2D3F70C32E8F2D807F803219F02B
:10244000C29480EFC822882089F081E0881609F4C0
:1024500068C0DD2009F472C0BB2009F468C0F8012F
:10246000858180FFC5CF8F70858361C02091A201D7
:1024700022FD35C0DD2069F1CC2039F08091960134
:10248000C82AC09296010E94250780E00E94E80AAF
:10249000292D2850330B2430310510F40E94EB0312
:1024A000AA2009F469CC8091940180FD65CCF801E3
:1024B00012828595859585950E943F08C8010E94E6
:1024C000AA0E809194018595859585950E941608A0
:1024D00053CC80E00E946108CC20D1F29DCFDD205A
:1024E00099F0909197018C2D892BB11003C00E9417
:1024F0005708CECFE1E0BE12FACF22FFC9CF98171E
:1025000039F280939701C4CFB11006C00E9418071A
:102510008C2D0E945008BCCFF1E0BF1609F4B8CF53
:10252000F5CFDD2031F025E02B1508F4B1CF8C2D4F
:10253000DECF34E03B1508F4ABCFEACFBB2041F34C
:10254000F9E38F1209C02FEF37EE83E021503040BE
:102550008040E1F700C000008E2D0E94610898CFF6
:102560008F2D86958695837061F0813009F090CF2C
:10257000C7019370D11002C090E080E00E94BF03B9
:1025800087CFC7019370D11002C090E080E00E9415
:10259000D5037ECF8E2DDD2029F00E94DA040E9423
:1025A000F80376CF0E941F04FACF8F2D837091F528
:1025B000D1106ECF4E2D429546954770440F440F73
:1025C0008E2D8F70042E01C0880F0A94EAF72E2DED
:1025D0002071E4FE07C02FE030E001C0220F4A95D1
:1025E000EAF720953F2D369536953370323069F0F5
:1025F00050F440919801313029F0822B84230E94BD
:102600004B0846CF842B822BFACF282B8091980140
:102610008227F5CF8695DD2011F08F2D81708823DC
:1026200009F436CF4E2D429546954770440F440F1E
:102630008E2D8F70042E01C0880F0A94EAF72E2D7C
:102640002071E4FE07C02FE030E001C0220F4A9560
:10265000EAF720953F2D369536953370323069F084
:1026600050F440918702313029F0822B84230E945C
:1026700005080ECF842B822BFACF282B809187025E
:102680008227F5CF9F2D9F70F92EDD2029F0892F0D
:102690000E943F088E2D2BCF8E2D0E9450088F2D2B
:1026A0000E941608F5CE8E2DE2EF8E16B1F1E815D8
:1026B00070F0F0EF8F16D1F021EF821691F0DD204F
:1026C00009F45EC0B11094CE8F2D8F712AC033EF04
:1026D000831651F194EF8912F2CF8091A20182FD0D
:1026E0002FC08F2D8F71DD20D9F21BC0DD2081F02E
:1026F000E4E0EB1508F4CCCE2F2D2F7181E090E0B3
:1027000001C0880F2A95EAF7909187028927AFCFF9
:10271000F5E0FB1508F4BCCEEFCF8F2D8F71D110F3
:10272000BFCF0E943F08B4CE80E0DD2009F49FCFE8
:102730009F2D9F7181E001C0880F9A95EAF797CF8E
:10274000DD2099F02F2D2F71F22E822F0E943F084D
:102750008091A20182FF07C038E0F39EC0011124DE
:102760008360809394018F2DDCCF81E00E94230849
:1027700081E08B1508F08CCE82E00E94230888CE81
:10278000BB2059F0893309F0E7CE9FEFE7EEF3E085
:102790009150E040F040E1F7DDCE8F2D8F7180CF7A
:1027A000F0E1EF16FFE5FF0609F4FFCB21E1E216A9
:1027B0002FE5F20609F4FDCB93EFE9169CE5F90647
:1027C00009F463CC08F0F7CBF8EDEF16FCE5FF0653
:1027D00009F457CC29EDE2162CE5F20609F461CC98
:1027E00037EDE3163CE5F30609F0F6CB26E241EEC1
:1027F00061EEC8010E949C0B0ACB30E1E3163FE575
:10280000F30609F4CCCB91E1E9169FE5F906A1F6B0
:1028100082E0C6CB85E0DE01119601900D928A958B
:10282000E1F7F801228189819A812111A9CA0E94C8
:102830007F07F82EADCAF6E1EF16FCE5FF0609F0BA
:102840006CCD8091520181114FCD89E20E944F07DA
:102850004ACC2AE5E2162DE5F20609F4A6CD78F475
:10286000E1148CE5F80609F441CD9EEDE9169CE5EE
:10287000F90609F052CD0E943F0E0E94290EECE5A8
:10288000EE16EDE5FE0609F43FCD08F490CD27EAFB
:10289000E2162DE5F20689F340CD1F93CF93DF9327
:1028A00080916101807F09F049C080915E01882399
:1028B00009F444C080919301D091620160915C0160
:1028C00070915D01A0915F01B0916001C62FC72397
:1028D00016E0D81799F190E0109711F0CF3F19F456
:1028E00001968770F6CF189F9001199F300D112423
:1028F000F901ED59FE4F41814713F2CF4081461354
:10290000EFCF42814111ECCF438154814A1B5B0BD5
:10291000483C510528F7809161018F708061809358
:102920006101F901E859FE4F80818F7080618083D9
:102930008CE591E00E94AA0E0E947507DF91CF916D
:102940001F910895A1E1B0E0E8EAF4E10C94DB1AEC
:102950008C0185E0F801DE011D9601900D928A95AB
:10296000E1F7F801E2808CE5A82E81E0B82E6091B5
:102970005F01709160016115710509F426C19091A4
:102980005C0140915D01892F84238F3F09F41DC1B3
:1029900020813181C380D480F0905E01F601E61B76
:1029A000F70BFF2009F4DCC080916101582F507FA4
:1029B000E83CF10508F09FC051116BC0FE2C431399
:1029C00014C0921312C0E11010C08F708061809308
:1029D0006101C5010E94AA0E80916101F801858301
:1029E0008F2D6196EAE00C94F71AC114D10429F0F6
:1029F000822F83238F3F09F003C180E0F82FF1700D
:102A0000DF2E80FF3CC0809193014091620156E02F
:102A1000841315C02D873E878D859E850E94180DD5
:102A2000292F22952F702230F0F0243018F59F7056
:102A3000F1F0F8019581907FD1F4D12C1EC090E087
:102A4000589FF001599FF00D1124ED59FE4F6181FF
:102A5000361306C06081261303C06281E6120FC0E0
:102A600001968770D5CF9F7011F0882331F3805E77
:102A7000883018F3C8010E94AA0EFD2CB1CFEE20B9
:102A800009F4AECF80916101816080936101F12CE6
:102A9000A7CF431306C0921304C0F801EE2009F437
:102AA00079C0C8010E94250D882309F1EE20F9F0B4
:102AB00080916101803270F020915C0130915D0164
:102AC00038872F831986DB86CA868C87CE010796C6
:102AD0000E94AA0E86E0F801ACE5B1E001900D92EB
:102AE0008A95E1F70E944D14FF24F39479CFC80131
:102AF0000E94AA0EF9CF51110AC08CE591E00E9404
:102B0000AA0E86E0F50111928A95E9F7C0CF43132A
:102B10000FC092130DC0E1100BC0F8018583C801EE
:102B20000E94AA0E86E0F50111928A95E9F758CF26
:102B3000C8010E94250D8823D1F2EE20C1F28091B8
:102B40006101803238F220915C0130915D013A835D
:102B500029831B82DD82CC828E83CE010196B8CF81
:102B6000E83CF105F8F6FE2CEE2009F243131FC0F5
:102B700092131DC08091610180FD10C0982F907F3D
:102B800069F0F8018583903F31F0982F907F905F36
:102B90008F70892B8583C8010E94AA0E86E0F801F8
:102BA000ACE5B1E001900D928A95E1F719CFC8012B
:102BB0000E94250D81118ECF8091610181608093EB
:102BC0006101C8010E94AA0E0BCFEE2009F48FCF3D
:102BD000C8010E94250DF82E882309F488CF86E0CD
:102BE000F801ACE5B1E001900D928A95E1F7809192
:102BF0005C0190915D010E94180D0E944D14F0CE71
:102C000081E08E25FBCEA7E1B0E0E9E0F6E10C948F
:102C1000E21A4B8B5C8B6D8B7E8B8F8B61111092CC
:102C200095011A8A198A85E0FE017396DE011D96C8
:102C300001900D928A95E1F786E0FE013D96DE0156
:102C4000179601900D928A95E1F7CE0107960E94A2
:102C5000A214811112C086E0FE013796DE011196A2
:102C600001900D928A95E1F78A859B85892B29F041
:102C700088859F8189238F3F81F516E0809193019C
:102C800090916201891317C06796E3E00C94FE1AD5
:102C900096E0929FD001939FB00D1124AD59BE4F85
:102CA000FE01319601900D929A95E1F780936201B1
:102CB0000E947507E2CF819FC00111248D599E4F5C
:102CC0000E94A214882301F38091930190E0019661
:102CD0008770992780939301D1CF2091620130E0D2
:102CE000C9010196877099274091930148171906E9
:102CF00079F60E941D0E109262011092930186E0F7
:102D0000ECE5F1E0DF011D928A95E9F7B6CF789402
:102D10001F921FB61F9211248F939F93AF93BF935F
:102D20008091C6019091C701A091C801B091C901DD
:102D30000196A11DB11D8093C6019093C701A09378
:102D4000C801B093C901BF91AF919F918F911F901E
:102D50001FBE1F9018951F921FB61F9211248F93AC
:102D60009F93AF93BF938091C401811113C0809151
:102D7000C6019091C701A091C801B091C9014196C7
:102D8000A11DB11D8093C6019093C701A093C801F6
:102D9000B093C901BF91AF919F918F911F901FBEBA
:102DA0001F901895CDB7DEB760970FB6F894DEBFC9
:102DB0000FBECDBF0E94B3039093B0018093AF01CB
:102DC00080E890E00FB6F8948093610090936100E2
:102DD0000FBE84E395E09093490180934801809170
:102DE0006900886080936900E99A8BE4809394027B
:102DF0008093C9028093A0028AE580939302809316
:102E0000C80280939F02539A80E0815009F0BBC0B2
:102E10005398789482E084BD93E095BD9AEF97BD76
:102E200080936E000E94450D811102C00E94800CAB
:102E30000FE311E0B4E4EB2EB1E0FB2EF801819139
:102E40008F018F3F11F00E943605E016F106B1F7B1
:102E500080E60E94360581E60E94360582E60E94E1
:102E6000360583E60E94360585E0EAEAF1E0DF01F7
:102E7000282F1D922A95E9F7ECE9F1E0DF011D9278
:102E80008A95E9F790E080E00E94331B883E9E4FD0
:102E900021F40E94450D811102C00E943F0E82E084
:102EA00090E00E942B1B8093A3010E945E0D9093E3
:102EB000A2018093A1010E946C0DEFE3FCE9319720
:102EC000F1F700C000000E946C0D8091AA0180FF04
:102ED00008C06FEF7FEF90E080E00E94571B0E94D8
:102EE0008F0383E090E00E942B1B0E944B0880E040
:102EF00091E09093C1018093C001FFEF20E732E0A1
:102F0000F15020403040E1F700C00000EE24EA9488
:102F100044E0242E53E0352E69E3462E70E1572E0F
:102F2000E9E06E2EFF24F394FFEA8F2EF1E09F2E4E
:102F3000ACE07A2E8091AE021091C501882359F140
:102F40001092AE020E94B3039093B0018093AF0140
:102F5000112309F4CBC11092C5010E941D0E0E94DD
:102F6000EB038091C501882309F4C0C10E94BA080F
:102F70000E946C0DEAEAF1E08191811187C18E1601
:102F80009F06D1F7D7CFA895AFE9BFE01197F1F72A
:102F900000C000003ACF1111E9CF8091AF019091AC
:102FA000B0010E94A403069708F4A0C1F092C501E5
:102FB0000E94BA08DBCF9F5FDD0C943009F0C0C1DE
:102FC0000F5F1F4F0530110509F0B0C1EC86ED868B
:102FD0001E860E94B3038160782F988B8F874C8563
:102FE0005D856E8588890E940316C7C1F092BA017B
:102FF0001BC2F092BB0121C2F092BC0164C2F092EC
:10300000BD016AC2109253026092540202E512E0BE
:103010001CC180915302823009F451C18330C9F040
:10302000813009F03EC02FB7F8946091C6017091CD
:10303000C7018091C8019091C9012FBF0E94CC1A8D
:1030400060935402709355028093560290935702F6
:10305000DDCF8091AA01809354028091AB018093CF
:1030600055028091AC01809356028091AD0180930E
:1030700057028091AE0180935802C8CF80915302CD
:10308000823079F460915402709155028091560219
:10309000909157020E94CC1A86E290E00E94391B60
:1030A000B5CFE0925202B2CF4091550260915402E6
:1030B000809153020E94AC0C9827892798279093FF
:1030C000570280935602A2CF2091560230915702A8
:1030D0003227232732274091550260915402809174
:1030E00053020E94090C92CF0E942F0C8FCF509256
:1030F00053028CCF309253024092540287CF0091FA
:1031000053021091540210270127102732E5A32EF5
:1031100032E0B32EC0905502D12CC6018E5A9D4F7D
:103120006C01C80189539F4FAC14BD0409F46ECFE4
:103130000933A3E01A0750F40E942B1BF501848386
:103140000F5F1F4FBFEFAB1ABB0AEBCFD501149631
:103150001C92F6CF009153021091540210270127C0
:10316000102722E5A22E22E0B22EC0905502C00EFA
:10317000D12ED11CC80189539F4FC016D10609F426
:1031800045CF0933E3E01E0728F4D50114966C916E
:103190000E94391BBFEFAB1ABB0A0F5F1F4FEACF6C
:1031A0000E94F90B33CF2092530230CF009153028B
:1031B0001091540210270127102792E5C92E92E0A2
:1031C000D92EA0905502B12CF501EE5AFD4F5F01AA
:1031D000C8018796AC14BD0409F418CF003A110554
:1031E00058F40E942B1BD60114968C930F5F1F4F2F
:1031F000FFEFCF1ADF0AECCFF6011482F7CF009170
:1032000053021091540210270127102782E5A82E9F
:1032100082E0B82EC0905502C00ED12ED11CC8013C
:103220008796C016D10609F4F1CE003A110528F4AC
:10323000D50114966C910E94391BBFEFAB1ABB0AE3
:103240000F5F1F4FECCF0E94E30880919F0284FF25
:10325000FACF4FE952E068E0C8010E942D0A085FEA
:103260001F4FE2E002371E0781F780919F0284FF23
:103270000AC04FE952E060E090E080E00E942D0A31
:103280001092720257CE0E94E308EFCFF8949AB1E1
:103290005B9A892F8C608AB98BB187258BB9FFE740
:1032A00028E331E0F15020403040E1F700C0000059
:1032B0008BB187258BB99AB95B9878943BCE86E21F
:1032C00090E00E942B1B1092540210925502109213
:1032D0005602809357029ACE2B30310508F0C3C0B6
:1032E000FBC02B30310508F06FC0A7C00E94E30877
:1032F00080917C02882309F418C18091930284FF95
:1033000014C10E946C0D882359F08FB7F894409136
:10331000C6015091C7016091C8017091C9018FBF6A
:10332000EAEAF1E0A4EAB1E010E000E0302F819198
:103330002D91281709F444CE90E0DD24D39428275A
:10334000422F4D2109F437CE9F8338878D2191E09C
:1033500009F490E099870E94B3038160782F9B87DE
:103360008A874F81588569858B850E940316F801ED
:10337000EC55FE4F8081D826D08286E0E8EBF1E064
:10338000DE01119601900D928A95E1F71092BA0133
:103390001092BB011092BC011092BD018B819C81E7
:1033A000892B09F44AC08091B6019091B7010E941F
:1033B000A4039C019091B201992309F492CF253185
:1033C0003105D8F19F3F19F09F5F9093B2011B81A7
:1033D000112359F00E94BA049FEF11160CF491E0EA
:1033E000899F802D11248093BA011C81112359F0EB
:1033F0000E94BA049FEF11160CF491E0899F802D72
:1034000011248093BB013091BA013323B1F0209194
:10341000BB01222391F045EB3403C0011124992311
:1034200009F4E4CD9093BA0145EB240390011124F3
:10343000332309F4DECD3093BB018D819E81892B2E
:1034400009F44AC08091B4019091B5010E94A4038F
:103450009C019091B101992309F43ECF21353105AA
:10346000D8F19F3F19F09F5F9093B1011D81112307
:1034700059F00E9498049FEF11160CF491E0899F77
:10348000802D11248093BC011E81112359F00E94CC
:1034900098049FEF11160CF491E0899F802D112460
:1034A0008093BD013091BC013323B1F02091BD0167
:1034B000222391F045EB3403C0011124992309F430
:1034C0009BCD9093BC0145EB240390011124332341
:1034D00009F495CD3093BD0146E050E0BE016F5F29
:1034E0007F4F88EB91E00E941E1B892B61F4809135
:1034F000BA019091BB01892B9091BC01892B9091CD
:10350000BD01892B11F00E94F80386E0FE0131967F
:10351000A8EBB1E001900D928A95E1F70E94EB03D0
:103520009091A90189138093A9010E948D0A0E949C
:10353000E30880917C02882309F4FCCC80919F02EF
:1035400084FFF8CC80917202803209F0F3CCE091D4
:103550005202E150E33108F0A4CDF0E0E558F44E1A
:103560000C94C61A97FB072E16F4009407D077FD2B
:1035700009D00E940A1B07FC05D03EF49095819566
:103580009F4F0895709561957F4F0895EE0FFF1F2F
:103590000590F491E02D09946927962769277827EB
:1035A0008727782708952F923F924F925F926F92CC
:1035B0007F928F929F92AF92BF92CF92DF92EF92C3
:1035C000FF920F931F93CF93DF93CDB7DEB7CA1B44
:1035D000DB0B0FB6F894DEBF0FBECDBF09942A886F
:1035E000398848885F846E847D848C849B84AA8417
:1035F000B984C884DF80EE80FD800C811B81AA81A4
:10360000B981CE0FD11D0FB6F894DEBF0FBECDBF6E
:10361000ED010895AA1BBB1B51E107C0AA1FBB1FE8
:10362000A617B70710F0A61BB70B881F991F5A954E
:10363000A9F780959095BC01CD010895FB01DC01AF
:1036400004C08D910190801921F441505040C8F779
:10365000881B990B0895F999FECF92BD81BDF89A08
:10366000992780B50895A8E1B0E042E050E00C94BD
:103670005F1B262FF999FECF92BD81BDF89A019765
:1036800000B4021639F01FBA20BD0FB6F894FA9AAA
:10369000F99A0FBE08950396272F0E943A1B0E94A5
:1036A000391B252F0E943A1B242F0C943A1B01969C
:1036B000272F0E943A1B0C94391BDC01CB01FC0123
:1036C000F999FECF06C0F2BDE1BDF89A319600B47B
:1036D0000D9241505040B8F70895F894FFCFDE1195
:1036E000DE1119121912B012CA1248124812D5125C
:1036F000421353135313021809183E185418641830
:1037000074185118511851185118511877187A18FF
:0C3710007F18AA18D018D318D618FF187C
:10371C008C03BC0A560A880A830A8B03FF5A8182DF
:10372C0083E200E900EA00B500B600B700CD0083E3
:10373C0001CC008A0192019401210223022402256A
:10374C0002260227022A02B300B4006F0070003177
:08375C003097969460616263EE
:00000001FF
